S01900006F70656E626C745F73746D3332663035312E7372656303
S31508000000D80400208D180008E3050008DF10000852
S3150800001000000000000000000000000000000000D2
S315080000200000000000000000000000001F13000888
S3150800003000000000000000005B1400086B180008B0
S3150800004077180008C5180008D1180008D318000842
S31508000050D5180008D7180008D9180008DB180008B2
S31508000060DD180008DF180008E1180008E318000882
S31508000070E5180008E7180008E9180008EB18000852
S31508000080ED180008EF18000800000000F118000835
S31508000090F3180008F5180008F7180008F9180008FA
S315080000A0FB180008FD180008FF18000801190008C9
S315080000B003190008000000000519000800000000E8
S315080000C00020C043834908600020C0438249086075
S315080000D0704770B504000D001600200000F0DAF92C
S315080000E0FF2805D06019401E00F0D4F9FF2801D179
S315080000F0002014E0600A802189004843774909688E
S31508000100884206D12B0032002100734800F0E8F837
S3150800011005E02B00320021006E4800F0E1F870BDC2
S3150800012070B504000E00200000F0B4F90500A0190F
S31508000130401E00F0AFF9EDB2FF2D02D0C0B2FF2885
S3150800014001D1002005E00100C9B22800C0B200F0C4
S3150800015048F970BD80B5002000905F48006800210E
S31508000160C943884201D101202FE000985A494968BD
S3150800017040180090009858498968401800900098DF
S315080001805549C968401800900098534909694018AC
S3150800019000900098504949694018009000984E49C7
S315080001A089694018009000984B49C9694018009021
S315080001B00098C14300910098401C00906A460421AB
S315080001C046480068C030FFF784FF02BD00B500202E
S315080001D0424909680968401840490968091D0968BB
S315080001E040183E4909680831096840183B490968BA
S315080001F00C310968401839490968103109684018EE
S3150800020036490968143109684018344909681831AB
S315080002100968401831490968C0310968401800283A
S3150800022001D1012000E0002000BD80B52A48006801
S315080002300021C943884206D0274800F098F80028CC
S3150800024001D100200DE0234800680021C9438842F7
S3150800025006D0204800F08BF8002801D1002000E0E5
S31508000260012002BD1D480068704780B5CA05D20D39
S31508000270002A01D000200BE002688A4201D1012041
S3150800028006E0016080229200001D00F091F901202D
S3150800029002BD38B505000C000F48854208D10D4D42
S315080002A021002800FFF7E1FF002810D100200FE009
S315080002B00A480068844203D1074D08480468EFE7F6
S315080002C0280000F054F80028EAD1002000E02800B1
S315080002D032BD0000D8040020DC060020B016000855
S315080002E0F4B582B004000D001F00680A8021890059
S315080002F04843009020680021C943884207D10099E5
S315080003002000FFF7B2FF002801D100202EE0206868
S315080003100099884208D000992000FFF7BAFF040028
S31508000320002C01D1002021E02068281A2018061D7B
S31508000330029D00F052F9201D301A8021890088425A
S315080003400CD300988021890041182000FFF7A1FFEF
S315080003500400002C01D1002008E0261D2878307002
S31508000360761C6D1C7F1E002FE3D10120FEBDF8B55B
S3150800037007000124386800F08DF8C0B2FF2801D1C3
S3150800038000202DE000F02EF9342000F0A1F900F04D
S31508000390A2F9012803D100F031F9002020E0002558
S315080003A000E06D1C802D17D2386804216943401877
S315080003B00090042068433818466800F00EF93100AA
S315080003C0009800F046F9042801D0002404E00098BB
S315080003D00068B042E5D0002400F010F92000C0B251
S315080003E0F2BD70B504000D0028002100C0B2C9B2E4
S315080003F0884201D200204AE020002549097AC0B285
S31508000400884205D3544800782900C9B2884201D2E7
S3150800041000203CE000F0E6F8342000F059F900F03E
S315080004205AF9012803D100F0E9F800202FE020004E
S31508000430C0B200F057F806002800C0B200F052F823
S3150800044004002800C0B200F06AF801002000401835
S31508000450401E801B401C840A002500E06D1C2800F5
S31508000460210080B289B288420ED200F0B6F8ADB249
S315080004708020C0006843301800F0C7F80428EDD083
S3150800048000F0BCF8002002E000F0B8F8012070BDCA
S31508000490B016000838B50400002500E06D1CEDB262
S315080004A00D2D1DD200F099F82C48EDB20C216943A8
S315080004B040588442F2D32948EDB20C21694340588A
S315080004C02649EDB20C226A438918496840188442C5
S315080004D0E4D22248EDB20C214D434019007A00E0DF
S315080004E0FF2032BD38B50400002500E06D1CEDB2D2
S315080004F00D2D11D200F071F81848EDB20C216943A0
S315080005004018007A2100C9B28842EFD11348EDB2EB
S315080005100C214D43405901E00020C04332BD38B597
S315080005200400002500E06D1CEDB20D2D12D200F07E
S3150800053054F80A48EDB20C2169434018007A2100A4
S31508000540C9B28842EFD10548EDB20C214D43401996
S31508000550406800E0002032BD48170008B0160008C1
S3150800056080B500F0E4F801BD10B500F0F0F80028F9
S315080005701DD000F0FEF8002819D000F027F900F089
S3150800058075F90121012000F075FA00F0E4F8C0229F
S3150800059001008020800500F00BF8032000F0A2FA85
S315080005A000F0D9F8001D046800F0C3F8A04710BD94
S315080005B070B514000D00060005E0287830706D1C33
S315080005C0761C00F00AF82000441E80B20028F4D1F8
S315080005D070BD80B500F0DBF801BD80B500F0DCF831
S315080005E001BDFEE700B535480068000605D5344864
S315080005F03449086034483349086000BD2F4800680C
S31508000600802101432D480160704710B5040004207D
S31508000610B020000300F078F8C0B2042817D12748A4
S3150800062000680221014325480160284804602348E0
S3150800063000684021014321480160B020000300F012
S3150800064063F81E490968022291431C4A1160C0B228
S3150800065010BD38B505000C00042000200090B0201D
S31508000660000300F051F8C0B2042825D113480068E9
S31508000670012101431148016020002880B0200003B1
S3150800068000F042F8C0B2042810D1AD1C0095200035
S31508000690000C00990880B020000300F035F80749DF
S315080006A0096801229143054A116005E00349096872
S315080006B001229143014A1160C0B232BD10200240A6
S315080006C02301674504200240AB89EFCD1420024080
S315080006D00C490860704700B504200A480068C0073E
S315080006E001D501200CE007480068C00601D50220A4
S315080006F006E004480068400701D5032000E004200E
S31508000700C0B200BD0C20024010B504000420FFF75B
S31508000710E2FF02E0FFF7DFFF641EC0B2012801D145
S31508000720002CF7D1002C00D10520C0B210BD72B63E
S31508000730704762B6704780B5FFF7C2FC01BD80B549
S31508000740FFF7C7FC02BD80B5FFF7EAFC02BD80B51E
S31508000750FFF73CFD02BD80B5FFF784FD02BD80B5FD
S31508000760FFF7F8FC002801D1002001E0FFF75DFD46
S3150800077002BD80B500F0E9F901219020C00500F01E
S3150800078043FA012801D1002000E0012002BD80B50E
S31508000790642000F0B3F901BD80B500F0B2F901BDDF
S315080007A080B500F071FA00F09BFC00202349087020
S315080007B001BD80B5224800F0DEFC012805D10020E5
S315080007C01E4908701E4800F07FFA01BD704780B5C3
S315080007D01A4A1278002A02D1C9B200F09FFC00F02A
S315080007E06FFA01BD00B515480078002805D0022823
S315080007F007D004D3032806D007E0402006E00020EF
S3150800080004E0002002E0002000E0402080B200BDA5
S3150800081000B50A480078002805D0022807D004D376
S31508000820032806D007E0402006E0002004E0002068
S3150800083002E0002000E0402080B200BDD000002089
S315080008407009002080B500F032FA02BD80B500F0CC
S315080008500DF8114811490860002011490860052063
S315080008601049086000201049086001BD00200D49A4
S315080008700860704700B50B480068C00304D50A48ED
S315080008800068401C0849086000BD80B5FFF7F2FF04
S315080008900548006802BD00007FBB000014E000E0C8
S315080008A018E000E010E000E0B809002030B50400C8
S315080008B0002000250020002100200025644801684A
S315080008C00C200840002806D0042807D0082808D09D
S315080008D00C2823D025E07948206024E0774820605A
S315080008E021E05B480068F025AD03054058480168DB
S315080008F0C02040020840AD0CAD1C002802D170484B
S31508000900454309E06F4800680107090F491C6B4811
S3150800091000F0AEFC68430500256004E06B482060E3
S3150800092001E0664820604A480168F020084000094E
S315080009306549085C2168C140616045480168E02056
S31508000940C0000840000A6049085C6168C140A160AF
S3150800095051480068C00502D45D48E0600AE03C489A
S315080009600068400403D4A0684008E06002E0A0687C
S315080009708008E06048480068400602D4554820616F
S3150800098002E080200002206143480068C00602D4C5
S315080009904A48606101E0206860613F480068800756
S315080009A0800F002802D1A068A0611AE03A480068C2
S315080009B08007800F012802D12068A06111E036481F
S315080009C000688007800F022803D180200002A061FA
S315080009D007E0314800688007800F032801D13748AF
S315080009E0A0612D480068C02189020140002902D172
S315080009F0A068E06123E028480068C0218902014018
S31508000A0080204002814202D12068E06117E0224836
S31508000A100068C0218902014080208002814203D1FA
S31508000A2080200002E0610AE01B480068C0218902B4
S31508000A300140C0208002814201D12048E061164869
S31508000A400068000602D42148206200E0256230BD15
S31508000A500410024000B5C9B2002905D01E4909682C
S31508000A6008431D49086004E01B49096881431A4880
S31508000A70016000BD00B5C9B2002905D0174909684B
S31508000A8008431649086004E0144909688143134875
S31508000A90016000BD000000003010024000B5C9B278
S31508000AA0002905D00E49096808430D49086004E085
S31508000AB00B49096881430A48016000BD00127A00A3
S31508000AC000093D002C100240C0000020006CDC022A
S31508000AD0809FD500128000001410024018100240B2
S31508000AE01C10024000210449096803229143084367
S31508000AF0010001480160704700000140164908805E
S31508000B00704780B5FFF7C1FE1449096888421BD3B0
S31508000B1013480078002808D101201149087080215F
S31508000B204900104800F07DF807E000200C490870DD
S31508000B30802149000B4800F077F8FFF7A6FE064922
S31508000B40098840180549086001BD80B5802149001B
S31508000B50044800F069F801BDC0090020B409002066
S31508000B60C30900200008004870B5002200230024AD
S31508000B70002246E0012393400C681C409C423FD16A
S31508000B800B79012B02D00B79022B19D18368032428
S31508000B90150002267543AC40A343836083684C79ED
S31508000BA0150002267543AC401C43846083880124E3
S31508000BB09440A343838083888C7994401C43848023
S31508000BC003680324150002267543AC40A34303605B
S31508000BD003680C79150002267543AC401C43046073
S31508000BE0C3680324150002267543AC40A343C360BB
S31508000BF0C368CC79150002267543AC401C43C46013
S31508000C00521C102AB6D370BD00B502000020108A07
S31508000C1089B20140002901D0012000E00020C0B2BD
S31508000C2000BD89B28161704701857047F0B4002321
S31508000C300023D2B20B005B075B0F042463439A4080
S31508000C40130089B2CA1004246243821889B2CC10F0
S31508000C5004256C430419246A0F250E007607760FBF
S31508000C6004277E43B540AC43146289B2CA100424F3
S31508000C7062438218126A134389B2C9100422514387
S31508000C8040180362F0BC70470020C5490870002070
S31508000C90C34988640020B54908700020B449088013
S31508000CA00020BF4988700020BD494870704700B5CC
S31508000CB0BB480078002801D1002000E0012000BDD3
S31508000CC00020AA490870704780B50178FF2917D116
S31508000CD000F087F8A5480078012802D1102000F016
S31508000CE077F8AF484421405E012808DB01209F4978
S31508000CF00870AB484421415EB84800F052F801BD7F
S31508000D00A749097801294BD10178C92932D0CC29BC
S31508000D103FD0CF293AD0D0292FD0D12933D0D229C4
S31508000D202ED0F32917D0F4290FD0F5290AD0F629A1
S31508000D300ED0FA2912D0FC2913D0FD2914D0FE2989
S31508000D4015D029E000F0CBF8C4E700F0EAF8C1E7CF
S31508000D5000F0BBF8BEE700F00DF9BBE700F09DF820
S31508000D60B8E700F095F8B5E700F07BF8B2E700F0D1
S31508000D706BF8AFE700F034F9ACE700F052F9A9E7F1
S31508000D8000F010F9A6E700F07DF9A3E700F08DF969
S31508000D90A0E700F09FF99DE7202000F019F899E7F1
S31508000DA0ADE780B589B2FFF712FD01BD10B5002386
S31508000DB002E004781B19401C0C00611E002CF8D1B7
S31508000DC0DBB21360012010BD0020754948707047DA
S31508000DD0FE21734AD170724908710220644908805D
S31508000DE0704780B5FFF7F0FF01206D490870FF20B6
S31508000DF06B49C87000206A49087169480079102152
S31508000E000143674801710020654948716448407983
S31508000E1063494871FFF7E6FC61498871FFF7F8FCFA
S31508000E205F49C871FFF7F4FC80B2000A5C49087292
S31508000E3001205B49487201205949887208204C49AB
S31508000E400880FFF778FC01BD80B50020544908707A
S31508000E50FFF7BAFFFF205249C870012044490880AD
S31508000E6001BDFF204E49C87000204D4908714C4805
S31508000E7040784B4948710020494988710020484903
S31508000E80C87100204649087206203949088070470B
S31508000E9080B50020FFF79CFF01BDFF204049C870C0
S31508000EA087483F49886400203D49087100203C492D
S31508000EB0487100203A49887107203949C91C486099
S31508000EC0C91E08202A4908807047FF21344AD17074
S31508000ED0406833498864012025490880704710B561
S31508000EE00400FFF77FFC80B2401E6178884203DA6F
S31508000EF02220FFF76DFF13E0627892B22848816CD2
S31508000F007048FFF755FBFF202549C8702448806CB8
S31508000F1061784018224988646078401C1449088022
S31508000F2010BD10B50400FFF75DFC80B2401E617865
S31508000F30884203DA2220FFF74BFF16E0606818495B
S31508000F408864627892B21648816C5E48FFF730FB77
S31508000F50FF201349C8701248806C61784018104900
S31508000F6088646078401C0249088010BD2309002067
S31508000F702409002080B5FF21094AD170524A4168E8
S31508000F800748806CFFF712FF0549087100200449DD
S31508000F90487100200249887108204C49088001BD23
S31508000FA0E008002080B5FF204949C870002048495C
S31508000FB00871002046494871FFF714FC44498871B6
S31508000FC000204349C8710020414908720020404961
S31508000FD0487207203D49088001BD0000E30800204B
S31508000FE010B50400FFF7FEFB621C80B2411E3848AC
S31508000FF0806CFFF7A4FB002803D13120FFF7E8FE39
S315080010000EE0FF203249C870FFF7ECFB3049896CC7
S3150800101080B2401E08182E49886401202B49088092
S3150800102010BD10B50400FFF7DDFB80B2801E6178A5
S31508001030884203DA2220FFF7CBFE22E0FF2024496C
S31508001040C8700120214908806078002807D1FFF779
S3150800105086FB002802D13120FFF7BAFE11E0A21C58
S3150800106061781B48806CFFF76AFB002803D13120A2
S31508001070FFF7AEFE05E01648806C61784018144903
S31508001080886410BD80B541681148806CFFF75BFB2A
S31508001090002803D13120FFF79BFE05E0FF200C490D
S315080010A0C87001200949088001BD80B5FFF75CFAC0
S315080010B0FF200749C87001200449088001BD0000C7
S315080010C0C8180008E4080020E708002024090020C2
S315080010D0E008002080B53120FFF77AFE01BDFEE763
S315080010E000B587B0E12000020090002001900020A2
S315080010F0029000200390002005900C200490694679
S31508001100544800F00DF980214901524800F08AF947
S315080011100121504800F064F907B000BD70B506001B
S315080011200C00E4B2412C03DB7F214B4800F090F918
S315080011302000C0B200F075F8C0B2012803D08321A0
S31508001140454800F085F900250DE0FFF746FAADB2EF
S31508001150705D00F066F8C0B2012803D08C213E48C5
S3150800116000F076F96D1C28002100C9B280B289B258
S315080011708842EAD370BD10B50400384800780028C4
S3150800118013D1374800F03DF8012838D134480078A3
S31508001190002834D0FFF779FB32490860002032492D
S315080011A0087001202D49087029E02D482E49097834
S315080011B04018401C00F025F8012816D12A48007866
S315080011C0401C29490870284800782549097888422A
S315080011D015D12548027892B224492000FFF7E8F98C
S315080011E000201E49087001200AE0FFF74EFB1D4942
S315080011F009686431814202D200201849087000202B
S3150800120010BD10B504002021124800F015F9012878
S3150800121005D1104800F0FAF82070012000E00020FF
S3150800122010BD10B5040080210A4800F005F9002811
S3150800123001D100200CE0E4B2210089B2054800F093
S31508001240E1F88021034800F0F7F80028F9D00120DA
S3150800125010BD0000004400404C170008C5090020D6
S315080012602C090020BC090020C40900202D090020F3
S315080012700022030A8B420BD203098B4219D2430878
S315080012808B422ED2411A00D201465241104670476F
S31508001290FF2209023FD012068B4205D31212090219
S315080012A08B4201D31212090203098B4219D300E0BB
S315080012B0090AC3098B4201D3CB01C01A52418309DB
S315080012C08B4201D38B01C01A524143098B4201D389
S315080012D04B01C01A524103098B4201D30B01C01AB4
S315080012E05241C3088B4201D3CB00C01A524183082E
S315080012F08B4201D38B00C01A524143088B4201D35B
S315080013004B00C01A5241884200D3401A5241CFD2EC
S3150800131001461046704708B500F09EF808BDFEE77E
S31508001320F0B589B004000D000027002600212068CA
S315080013300121884320606168080036490140080099
S31508001340A9680143616021680800334901400B0020
S315080013506868EA6802432969114319432160A1684C
S3150800136008002E490140080069690143A1606846E2
S31508001370FFF79CFA2148844201D1069E05E02048E1
S31508001380844201D1079E00E0029E206800040CD525
S31508001390022070432968FFF76BFF070002204643C7
S315080013A030002968FFF764FF08E030002968FFF776
S315080013B05FFF070030002968FFF75AFF28684008D2
S315080013C0814200D37F1C2068000406D578084107AF
S315080013D0490F134838400F000743A78109B0F0BDED
S315080013E000B5C9B2002904D0016801220A43026087
S315080013F003E0016801229143016000BD0038014005
S3150800140000440040C905C90D01857047808CC00598
S31508001410C00D7047FFCFFFFFF3E9FFFFFFFCFFFF9B
S31508001420F0FF00008268034B134083608268114313
S3150800143081607047FFEFFFFF00B502000020D0690A
S315080014400140002901D0012000E00020C0B200BD03
S3150800145080B5FFF7C2F8FCE77047FEE780B5374866
S31508001460006801210143354801603548006835495F
S3150800147001403348016031480068334901402F482C
S3150800148001602E480068314901402C4801602C480B
S3150800149000682F4901402A4801602E4800680F213C
S315080014A088432C4908602C4800682C4901402A4882
S315080014B001602B48006801218843294908600020FB
S315080014C02849086000F001F801BD00B51120264939
S315080014D008601B4800681A490860194800681849D6
S315080014E008601748006821490140154801601448FA
S315080014F00068A02189030143114801600F4800686C
S315080015008021490401430D4801600C4800688001A8
S31508001510FBD50B4800680321884309490860084839
S3150800152000680221014306480160054800680C214D
S3150800153001400829F9D100BD000000000010024052
S31508001540041002400CB8FFF8FFFFF6FEFFFFFBFF92
S31508001550FFFFC0FF2C10024030100240ACFEFFFF18
S31508001560341002400810024000200240FF7FC0FFEE
S3150800157080B500F005F800F05BF800F067F8FCE7C6
S3150800158000B583B0012180200003FFF763FA01212B
S3150800159080208002FFF782FA012180208002FFF76F
S315080015A059FA802040000090012069460871002001
S315080015B06946887103206946487100206946C871E2
S315080015C069461A48FFF7D0FA802149001748FFF7FD
S315080015D02BFB00206946087100206946C871012066
S315080015E0009069469020C005FFF7BEFA0122022145
S315080015F09020C005FFF71AFB012203219020C005A1
S31508001600FFF714FB0C20009003206946487102205E
S315080016106946087100206946887101206946C871C3
S3150800162069469020C005FFF79FFA07BD00080048E5
S3150800163080B5FEF795FFFEF7CCFFFFF707F9FFF732
S315080016407AF8FFF7ADF800F00BF801BD80B5FEF7A4
S31508001650C4FFFFF70FF9FFF7ACF800F00CF801BD6F
S3150800166080B5012010490870FFF70FF90F49086087
S3150800167000F001F801BD80B5FFF7E4F8012811D0A4
S315080016800948007801280DD1FFF7FFF807490968CE
S31508001690FA2252008918884204D3002002490870A9
S315080016A0FEF762FF01BD0000C2090020B009002054
S315080016B000200008000800000400000000280008B8
S315080016C000080000050000000030000800080000BF
S315080016D006000000003800080008000007000000A7
S315080016E00040000800080000080000000048000844
S315080016F0000800000900000000500008000800006B
S315080017000A00000000580008000800000B0000004E
S3150800171000600008000800000C00000000680008CF
S31508001720000800000D000000007000080008000016
S315080017300E00000000780008000800000F000000F6
S31508001740008000080080000010000000433A5C5743
S315080017506F726B5C736F6674776172655C4F7065E8
S315080017606E424C545C5461726765745C536F757253
S3150800177063655C41524D434D305F53544D33324699
S31508001780305C756172742E630000000070B401212C
S31508001790002213E00468001D0C4202D04D466D1E5F
S315080017A064192260241D1B1F042BFAD225009E07EC
S315080017B001D52280AD1C0B4000D02A700368001D9D
S315080017C0002BE7D170BC704730B401210268001DB8
S315080017D0002A0FD00368C318446808300C4202D0A8
S315080017E04D466D1E64191D6825601B1D241D121F9C
S315080017F0ECD0F8E730BC704710B507497944183182
S31508001800064C7C44163404E0081D0A688918884783
S315080018100100A142F8D110BD080000002800000010
S315080018206DFFFFFFF0040000D80400200000000050
S3150800183099FFFFFF140000006C000000C0000020A4
S315080018400000000000F00BF8002801D0FFF7D4FFD5
S31508001850002000BF00BFFFF78BFE00F002F8012052
S31508001860704780B500F002F801BDFEE70746384626
S3150800187000F002F8FBE7FEE780B500BF00BF024AAA
S3150800188011001820ABBEFBE7260002000248854679
S315080018900248804702480047D80400205D14000823
S315080018A0B91800080000000001020304010203043D
S315080018B0060708090400000000BF00BF00BF00BFFC
S315080018C0FFF7C0FFFEE700004F70656E424C5400FC
S315080018D0FEE7FEE7FEE7FEE7FEE7FEE7FEE7FEE7D2
S315080018E0FEE7FEE7FEE7FEE7FEE7FEE7FEE7FEE7C2
S315080018F0FEE7FEE7FEE7FEE7FEE7FEE7FEE7FEE7B2
S30B08001900FEE7FEE7FEE724
S705080018B921
